:020000040000FA
:100000008301532800000000F200030E8301F30077
:100010000B1183120313A80F0E28A90AAF0F112882
:10002000B00A730E8300F20E720E09008B138B1B45
:10003000162871088A0070088200000883160313CE
:100040009A001C158B138B1B222855309D00AA305B
:100050009D009C148B179C182B281C119B0A840A4A
:10006000F00B1D280800831603131C141A088000C7
:100070009B0A840AF00B3328080000308316031310
:100080009B0083130230F000203084001D20080004
:100090000030831603139B0083130230F0002030DE
:1000A00084003320080020308B008312031380303B
:1000B0008500003086008F30831681003F30850038
:1000C00000308600831207309F00831320308400A5
:1000D0008001840A841F682884168001840AF03015
:1000E0000402031D6D288317203084008001840AD8
:1000F00050300402031D7628482083120313810127
:100100000B118B1783120313A71C8828A3019628B1
:1001100083120313271F96282418962824142718BF
:100120009328A30A962883120313A30383120313AD
:10013000271B9B282410DD30F0000130F1008312D2
:1001400003130310230DF0070318F10A162083127E
:100150000313A500F00A0319F10A162083120313F2
:10016000A6008B172518B6280612B7280616A5185C
:10017000BB288612BC2886162519C0280613C1285C
:100180000617A519C5288613C6288617251ACA2852
:100190008611CB288615A51ACF280611D02806155A
:1001A000251BD4288610D5288614A51BD92806100F
:1001B000DA280614061AE028061CE3282714E32888
:1001C0008312031327100030831203132902031D27
:1001D000EB2814302802031CF8280030A902143040
:1001E000A802031CA9032719F7282715F8282711A7
:1001F00083120313A71FFF28AA01AB011229831240
:100200000313271D12292C1812292C14A7190C29A5
:10021000AA0F1229AB0A122983120313AA032A0F69
:100220001229AB0383120313271917292C108312E9
:100230000313A711051C21292D1821292D14271678
:100240002729831203132712051827292D1083123B
:100250000313B21C2E29A001A1014129831203130B
:10026000271E41292E1841292E14A71A3B29A00F19
:100270004129A10A412983120313A003200F412918
:10028000A10383120313271A46292E108312031386
:10029000A7122008F0002108F100A71F55290030FF
:1002A000F1020030F002031CF10371088312031302
:1002B0002B02031D5D2970082A0283120313031CFD
:1002C0006329A7176429A713B1186E2931187A2951
:1002D000321C7A29AF01B001B11427170030831204
:1002E00003133002031D762904302F02031C7A29E0
:1002F000B110271383120313321C80293114832970
:10030000831203133110A71B872932108A29831205
:1003100003133214271A9029221C902922103D2001
:1003200083120313271E95292214073020028312FB
:100330000313031D9D29B2149E29B210321DA22958
:100340000517A5298312031305133219A929851747
:10035000AC29831203138513321EB029B301BE29C1
:1003600083120313271CBE293418BE293414B21972
:10037000BB29B30ABE2983120313B30383120313E9
:100380002718C329341083120313B211321ACA2951
:100390000230CB2902303302031CD0293216D12976
:1003A00032123308013C83120313031CDB290319A7
:1003B000DB293215DC293211822801340034023461
:1003C0000034043400340834003410340034203451
:1003D00000344034003480340034003401340034BC
:0A03E0000234003404340034083401
:084000000000010000000000B7
:02400E00183F59
:1042000000000000000000000000000000000000AE
:10421000000000000000000000000000000000009E
:10422000000000000000000000000000000000008E
:10423000000000000000000000000000000000007E
:10424000000000000000000000000000000000006E
:10425000000000000000000000000000000000005E
:10426000000000000000000000000000000000004E
:10427000000000000000000000000000000000003E
:10428000000000000000000000000000000000002E
:10429000000000000000000000000000000000001E
:1042A000000000000000000000000000000000000E
:1042B00000000000000000000000000000000000FE
:1042C00000000000000000000000000000000000EE
:1042D00000000000000000000000000000000000DE
:1042E00000000000000000000000000000000000CE
:1042F00000000000000000000000000000000000BE
:00000001FF
